:1000000039280F0000010F0000018928F528012878
:100010000F0000010F0000016928FD20D5B717056A
:10002000000013056510970500009385E5149308FB
:10003000100873000000170500001305050F73007A
:100040000000170500001305650E7300000017057A
:1000500000001305C50D7300000082801705000025
:100060001305850C970500009385850C93081008EF
:1000700073000000170500001305250B970500000D
:100080009385950B73000000170500001305050A02
:10009000970500009385E50A73000000170500002E
:1000A0001305E508970500009385350A73000000E5
:1000B000828017050000130525079705000093852A
:1000C0006509930810087300000017050000130568
:1000D000C505970500009385750873000000170596
:1000E00000001305A504970500009385C50773005C
:1000F0000000170500001305850397050000938590
:100100001507730000008280F32210C09102732350
:1001100010C073D000800F00000173500080E368AE
:1001200053FE8280310032003300340052494E4782
:1001300020434C4F00524F4144534544200020205F
:1001400020414E4F52540054202020482053540048
:1001500020464F4C20444554004C4F57204F555299
:1001600020002020202020202020002020202020CF
:0E017000202020002020202020202020000021
:00000001FF
